:1000000000308A00C12D00000A108A100A118207F0
:1000100028340C34013406340A108A100A1182077D
:100020005534643465346C3461346A347434653402
:10003000203470346134723400340A108A100A118A
:1000400082076B34723475346834753400340A10A6
:100050008A100A1182072034443465346A347434B7
:1000600065342034703461346B3475342034643436
:100070006F34203400340A108A100A118207703459
:1000800072346F34733474347234653464340034CD
:100090000A108A100A11820756347934733469348D
:1000A0006C3461346D3400340A108A100A118207EE
:1000B0004B3461346C346934623472346134633487
:1000C000653400340A108A100A11820754347234DD
:1000D00069346D3400340A108A100A1182075634CC
:1000E0007934733469346C346134743400343F309F
:1000F0008400000803198B280130A100A001A00B87
:100100007F28A10B7E284A30A000A00B8528000084
:100110000000800B7C28003406080F39C600450E0D
:10012000A000F030A0052008F0394604860006152E
:10013000831606110000831206118316061183121E
:100140000034C308031DA6288610A728861483162A
:1001500086108312C40E4408C5008C20C40E4408C7
:10016000C5008C200D30A000A00BB4280034143042
:10017000BF0077200F308316860583128610831602
:10018000861083120611831606118312B6013608F3
:10019000023C031CD3280230BF0077200330C50087
:1001A0008C20B60AC7280D30A000A00BD52802303D
:1001B000C5008C200D30A000A00BDC28B60136084D
:1001C000023C031CEF2836080420B700C30137089F
:1001D000C400A1200230BF007720B60ADF288A11B0
:1001E000022EA51025088316870083128714251078
:1001F00025088316870083120714B6013608073CCA
:10020000031C16292512250883168700831207125E
:10021000A51125088316870083128715A5112508C7
:100220008316870083128711B60AFE28A5102508B9
:1002300083168700831287102510250883168700F0
:1002400083120710A51125088316870083128715CE
:1002500083168611831286158A11032EBE013E086D
:10026000073C031CE429A510250883168700831288
:100270008710251225088316870083120712BD01F7
:100280003D08073C031C5229A51125088316870049
:1002900083128715A51125088316870083128711FD
:1002A000BD0A4029251225088316870083120716E8
:1002B000A51125088316870083128715A511250827
:1002C000831687008312871125122508831687005D
:1002D00083120712BD013E083D0203187D29A511B6
:1002E00025088316870083128715A5112508831614
:1002F000870083128711BD0A6B29A5102508831674
:100300008700831287148316861183128611831641
:10031000861183128615BD013D08043C031C9E29ED
:10032000A51125088316870083128715A5112508B6
:100330008316870083128711BD0A8C29251525088D
:10034000831687000030831207190130013C031D1A
:10035000AC293E08A100E629A511250883168700CF
:1003600083128715A511250883168700831287112C
:1003700025152508831687000030831207190130E0
:10038000013C031DC7293E080838A100E629A51134
:1003900025088316870083128715A5112508831663
:1003A00087008312871125152508831687000030E2
:1003B000831207190130013C031DE2293E08103861
:1003C000A100E629BE0A2F298030A1000034A51122
:1003D00025088316870083128711251025088316A8
:1003E000870083120710BC013C08073C031C1A2A33
:1003F0003B08A0003C08A1000319022A0310A00C2E
:10040000A10BFE292018062A0712072A0716251213
:100410002508831687008312A511250883168700F7
:1004200083128715A511250883168700831287116B
:10043000BC0AF429251025088316870083120714A7
:100440002510250883168700831207100034013019
:100450003F02C1004008023C031D302A4030C10762
:1004600041088038C200C3014208C400A120003402
:100470003E08A0000C30200203194B2A0A3020024B
:100480000319532A0D3020020319592A083020027B
:1004900003195E2A632AC3010130C400A12002307F
:1004A000BF0077206F2A0130BF000230C000272232
:1004B0006F2A0130BF00C00027226F2AC30110300D
:1004C000C400A1206F2A3E081F3C031C692A073084
:1004D000BE050130C3003E08C400A1206F2A0034CD
:1004E0000830A1001F08C73921049F000330A00075
:1004F000A00B782A3D0884001F151F197D2A1E08AD
:1005000080000030A1001F08C73921049F0003307C
:10051000A000A00B892A3E0884001F151F198E2AEF
:100520001E08800025172508831687008312071BE5
:10053000AA2AA630A000A00B9B2A00002517250898
:10054000831687008312071BA92A3F088400013005
:100550008000AD2A3F0884008001A5172508831676
:1005600087008312871BC52AA630A000A00BB62ADD
:100570000000A5172508831687008312871BC42A4D
:100580004008840001308000C82A400884008001AF
:100590000034BE08031DCE2A8712CF2A8716A51263
:1005A00025088316870053308312A000A00BD62A9B
:1005B000BE080319DD2A8712DE2A8716A512250830
:1005C0008316870053308312A000A00BE52A003465
:1005D0001F30BA05390EA000A00DE030A00520089C
:1005E000BA04BA0E3A080F39BC00BA0E3A080F39ED
:1005F000BC07BC0ABE01C9220830BB00BB080319F6
:100600000B2B0030BA1B0130BD00BE00C922031005
:10061000BA0DBB03FE2A0430BB00BB0803191A2B1A
:100620000030BC190130BD00BE00C9220310BC0D52
:10063000BB030D2BA512250883168700831287168E
:1006400000343A308400FC308005800C800C0008B7
:1006500003192E2B2C2B0000800B2B2B8A11452DE0
:100660000330B600B7012E212108B8003808073C36
:10067000031D3B2BB60A38080F3C031D402BB60365
:100680003608033C0318462B0130B600B608031D9C
:100690004B2B0330B6003808163C031D5E2D01308D
:1006A0003607A1000130A000A10803195B2B03103D
:1006B000A00DA10B572B20080138BA00BB00E72181
:1006C00001303602FD3E03184E2D033EB32D80301F
:1006D000AB00AA00A900A800A700A6000C30BE002D
:1006E0003822BD013D080C20BD0ABE0038220C3066
:1006F0003D02031D722B0130BF000230C0002722D3
:10070000BD013D081D20BD0ABE00382205303D0256
:10071000031D812B25172508831687008312071FC9
:10072000B92B2E212108173C031D972BBD2C3930E6
:10073000BD003A30BE003B30BF003C30C0007022EC
:10074000390827020318A62B3908A7002608390202
:100750000318AC2B3908A6003A0829020318B22B5B
:100760003A08A90028083A020318B82B3A08A8004A
:100770008A2B0230BD00FA30BF007720BD0BBB2BA7
:100780000C30BE003822BD013D082720BD0ABE0046
:1007900038220F303D02031DC42B0130BF00023050
:1007A000C0002722BD013D083B20BD0ABE00382203
:1007B00008303D02031DD32B25172508831687001B
:1007C0008312071FED2B2A30BD002B30BE003B30BB
:1007D000BF003C30C0007022DC2B2A082702AC008E
:1007E00026082A02AD002B082902AE0026082A029C
:1007F000AF00AC0CAC0CAC0C1F30AC05AD0CAD0CB0
:10080000AD0CAD05AE0CAE0CAE0CAE05AF0CAF0C26
:10081000AF0CAF0503178D018F0103132C080317CD
:100820008C0083168C130C15831203130B08A00085
:100830008B138316031755308D00AA308D008C144E
:100840008C18202C0C118312031320088B04013008
:1008500003178D008F0103132D0803178C008316D7
:100860008C130C15831203130B08A0008B13831633
:10087000031755308D00AA308D008C148C183E2C37
:100880000C118312031320088B04083003178D000A
:100890008F0103132A0803178C0083168C130C1581
:1008A000831203130B08A0008B1383160317553014
:1008B0008D00AA308D008C148C185C2C0C118312C6
:1008C000031320088B04093003178D008F010313D5
:1008D0002B0803178C0083168C130C15831203133B
:1008E0000B08A0008B138316031755308D00AA3018
:1008F0008D008C148C187A2C0C1183120313200891
:100900008B04023003178D008F0103132E08031789
:100910008C0083168C130C15831203130B08A00094
:100920008B138316031755308D00AA308D008C145D
:100930008C18982C0C118312031320088B0403309D
:1009400003178D008F0103132F0803178C008316E4
:100950008C130C15831203130B08A0008B13831642
:10096000031755308D00AA308D008C148C18B62CCE
:100970000C118312031320088B044E2D0630B9008E
:100980000130BA00E8220130B9003008BA00E8228C
:100990000230B9003108BA00E8224E2D03178D014C
:1009A0008F0183168C130C1483120C080313AC00F4
:1009B000013003178D008F0183168C130C148312E2
:1009C0000C080313AD00083003178D008F01831648
:1009D0008C130C1483120C080313AA00093003179C
:1009E0008D008F0183168C130C1483120C080313D3
:1009F000AB00023003178D008F0183168C130C148B
:100A000083120C080313AE00033003178D008F010F
:100A100083168C130C1483120C080313AF00C83018
:100A2000BF0077200630BF000230C0002722B90186
:100A300039084820B90ABE00382207303902031DA0
:100A4000182D2E212108803C031D4D2D3030BD0076
:100A50003130BE003230BF003330C0007022B00CE5
:100A6000B00CB00C1F30B005B10CB10CB10CB1051D
:100A70000130B9003008BA00E8220130BF00772009
:100A80000330B900BA30BA00212BB90B422D023025
:100A9000B9003108BA00E822212D4E2D0130360769
:100AA000A1000130B900A10803195A2D0310B90D96
:100AB000A10B562D3908BB00E721B70137083602D4
:100AC0000319B02D3608B7000C30BE0038220130B3
:100AD0003602FD3E03189E2D033EBA2D0530BF00A1
:100AE0000230C0002722B90139085420B90ABE00DB
:100AF000382209303902031D742D9E2D0730BF00A6
:100B00000230C0002722B90139086220B90ABE00AC
:100B1000382204303902031D842D9E2D0630BF007B
:100B20000230C0002722B90139086B20B90ABE0083
:100B3000382207303902031D942D9E2D01303607CF
:100B4000A1000130B900A1080319AA2D0310B90DA5
:100B5000A10BA62D3908BB00E721FA30BF00772092
:100B6000332B8A11042E0A148A100A158207672B68
:100B7000BE2CCE2C0A148A100A1582076E2D7E2DEB
:100B80008E2D84011F308305073083169F00FF30B0
:100B90008312A500043083169F0083121F08383982
:100BA00001389F009412A51225088316870083122E
:100BB00025162508831687008312A511250883169C
:100BC0008700003083129400831694008312A001E2
:100BD000A01DF22D07308101813084000008C0394A
:100BE0000F3880006400813084000008C039200480
:100BF000800090010030A100920000308316920026
:0C0C00008312B728F128302B042E63006B
:02400E00F13F80
:00000001FF
